:1000000033C0000046C0000044C0000042C00000F1
:1000100040C000003EC000003CC000003AC00000EC
:1000200038C0000036C0000034C0000032C00000FC
:1000300030C000002EC000002CC000002AC000000C
:1000400028C0000026C0000024C0000022C000001C
:1000500020C000001EC000001CC000001AC000002C
:1000600018C0000016C0000011241FBECFEFD8E05A
:10007000DEBFCDBF11E0A0E0B1E0E2E3F5E102C0F8
:1000800005900D92A230B107D9F70E947C090C941B
:10009000970AB6CFBF92CF92DF921F93CF93DF9391
:1000A000DC01CB01142FE901E4E3F8E30F921F9286
:1000B0007EEF6AE659E544E8D92EC82EBA2E212FE4
:1000C0001D2E0C2E09952131F9F71F900F90DF910D
:1000D000CF911F91DF90CF90BF900895BF92CF92A4
:1000E000DF921F93CF93DF93DC01CB01142FE90143
:1000F000E4E3FFE30F921F927EEF6AE659E544E8DE
:10010000D92EC82EBA2E212F1D2E0C2E0995213145
:10011000F9F71F900F90DF91CF911F91DF90CF9053
:10012000BF900895CF93DF93FA01E901213831059B
:1001300010F0C0E8D0E0AB01BC0140789E01CF01D7
:100140000E947309CE01DF91CF9108952F923F92C3
:100150004F925F926F927F928F929F92AF92BF92D7
:10016000CF92DF92EF92FF920F931F93CF93DF9383
:100170004A01E9012138310510F0C0E8D0E01E0144
:10018000369427946B017C0120E8C222D40180E0E0
:1001900090E060E070E082159305B9F0F601E8198F
:1001A000F909EA0FFB1F259134914D915D912417B8
:1001B000350709F071E040955095422B532B4F3F86
:1001C0005F4F09F061E00196E6CF772351F1662396
:1001D00039F020E030E043E0C701B601F8010995AD
:1001E00026013701A12CB12CA214B30491F0F40123
:1001F000219131914F0141E0C301B201F80109950C
:10020000F2E04F0E511C611C711C2FEFA21AB20AB2
:10021000EBCF20E030E045E0C701B601F8010995D9
:1002200002C0C0E0D0E0CE01DF91CF911F910F91CD
:10023000FF90EF90DF90CF90BF90AF909F908F9006
:100240007F906F905F904F903F902F9008950F9305
:100250001F93682F70E080E090E048E08B019C01E4
:10026000369527951795079560FF0BC0C901B80112
:1002700050E2652753E8752758EB85275DEE9527F3
:1002800002C0C901B801415049F71F910F9108956B
:10029000CF92DF92EF92FF92C72ED82EE92EFF2445
:1002A000842F8627D4DF6C257D258E259F25FF9002
:1002B000EF90DF90CF90089528E088E190E00FB6AE
:1002C000F894A895809360000FBE20936000A895D5
:1002D000F894D8E0CEEF28E3299320E0299314BEC8
:1002E000FFCF8FEF08951DC4000066C4000040C416
:1002F00000003EC400003CC400003AC4000038C402
:10030000000036C4000034C4000032C4000030C411
:1003100000002EC400002CC400002AC4000028C421
:10032000000026C4000024C4000022C4000020C431
:1003300000001EC400001CC400001AC4000018C441
:10034000000016C4000014C4000012C400007E3F68
:10035000F9F76A36F9F75935F9F74438F9F7EC2D1A
:10036000FD2DB7B6B0FCFDCF27BFE895B7B6B0FC02
:10037000FDCF21E1B7B6B6FCF4CF0895FFFFFFFF34
:10038000FFFFFFFFFFFFFFFFFFFFFFFFFFFFFFFF7D
:10039000FFFFFFFFFFFFFFFFFFFFFFFFFFFFFFFF6D
:1003A000FFFFFFFFFFFFFFFFFFFFFFFFFFFFFFFF5D
:1003B000FFFFFFFFFFFFFFFFFFFFFFFFFFFFFFFF4D
:100A80005553426173704C6F616465722076302EED
:100A900039372E312C206279205374657068616E6D
:100AA0002042616572776F6C6620286D617472698F
:100AB0007873746F726D40676D782E6465292C2091
:100AC00053636877616E736565203230313400009E
:100AD0000902120001010080320904000000000038
:100AE000000012011001FF000008C016DC05020121
:100AF000010200010E035500530042006100730023
:100B000070001C037700770077002E0066006900F4
:100B10007300630068006C002E006400650004032D
:100B2000090411241FBECFEFD8E0DEBFCDBF24B72C
:100B3000D8E0CEEF39913833399109F03FEF309357
:100B40003E0120933D0111E0A0E0B1E0EAEFFFE7B4
:100B500002C005900D92A630B107D9F721E0A6E0BA
:100B6000B1E001C01D92AD33B207E1F781D1B6C348
:100B7000BACBDC018FEF9FEF332715C02D912827CB
:100B8000722F22952727822F269526952827239591
:100B90002270321777952795822F8927972F769580
:100BA000279597278227615048F78095909508955B
:100BB000E0DF8D939D930895CF93CFB7CF93DF93CD
:100BC000C3954F9BE9F74F9B0BC04F9B09C04F9BB1
:100BD00007C04F9B05C04F9B03C04F9B01C089C0FE
:100BE0006F93C0912001DD27C95DDE4F2F9365E52E
:100BF0004F9B03C02F916F91E6CF0F931F934F939D
:100C000020E040E15F9309B1047807FB27F93F93A7
:100C100050E03BE039C0147840642F77012F5F5FCC
:100C20001EC0406819B114782F7752501FC040641D
:100C300009B12F770478D1F15F5F00C023C0406213
:100C400019B12F77147891F15F5F00C025C0047847
:100C50001027515012F45D5F0000115027952C3F72
:100C600019B1C8F614780127015027952C3FC8F612
:100C70004227499309B1047810274F7311502795E3
:100C80002C3FA8F64695469519B1147879F00127BE
:100C9000015027952C3F98F66B5A60F3315009B1FB
:100CA000B0F600C011E01CBB002717C03B503195C7
:100CB000C31BD04011E01CBB0881033CF9F00B348E
:100CC000E9F020911E011981110F1213EDCF0936A1
:100CD00051F10D3211F0013E39F7009325013F919A
:100CE0005F914F911F910F912F916F91CCB3C0FDE8
:100CF00067CFDF91CF91CFBFCF911895209125017C
:100D0000222369F310912301112339F534303AF18C
:100D10003093230120931F01109120013BE0311BF0
:100D2000309320011CC0009123010130B4F40AE586
:100D30003091010134FD14C000930101C3E1D1E001
:100D400013C0052710E000C000000BB91AC005272A
:100D500010E0221F1DC010E021C04AE502C032EDA4
:100D6000432FC4E1D0E032E01AB114685F9A0BB1AE
:100D70001AB954E820E865E320FF05270BB9279549
:100D800017951C3FF0F66695B8F7B1F720FF0527D9
:100D90000BB9279517951C3FD0F62795179517FF88
:100DA000052700001C3F0BB9B0F629913A9519F7B9
:100DB0000B7710912401110FC651D0400BB911F0DF
:100DC00010931E0111E01CBB00681AB11B77402F65
:100DD0004B7754E05A95F1F70BB91AB94BB97FCF5D
:100DE000FC013381932F4481842F2281203339F4F5
:100DF0004370E42FF0E0EE5FFE4F808108952835C8
:100E000029F431110EC0E1E0F0E006C0203599F47C
:100E100031110CC0E0E0F0E089E08093570084914C
:100E20000895383019F5E3E0F0E0F6CF3830F1F40A
:100E3000E2E0F0E0F1CF203221F4FC01EE0FFF1FE1
:100E400006C0283231F4FC01EE0FFF1F3196849169
:100E50000895203A09F42CC2203C19F4658130D25F
:100E600005C02F3F19F481EF8093110180E00895B0
:100E70001AB880E48BB981E085BF82E085BFE0E0ED
:100E8000F1E7A89531978040E1F780913D01877F98
:100E900021F480913E01882381F04E9B0EC0F8948E
:100EA000579A1BB81DBA1092690081E085BF15BE24
:100EB000E0910A01F0910B0109958EEF80931101E9
:100EC00014BE88E10FB6F894809360001092600021
:100ED0000FBE80916900826080936900E89A579AFA
:100EE0008CE0E0E0F5E3A89531978040E1F7579872
:100EF000789480912301835087FD46C19091200111
:100F0000CCE0D0E0C91BD109C95DDE4F90911F0133
:100F10009D3209F0B9C0883009F034C183EC809368
:100F200013018AE580930101109212014881842FF8
:100F3000807639818823B9F186E091E0909322018F
:100F400080932101333031F4CE014ADF80930901CF
:100F500024E090C0353019F13A3009F18CEF830F5D
:100F6000863098F48A819B819093100180930F01C1
:100F70003930B9F08E8180930E018D81827080931B
:100F80000D0130930C012FEF6FC0809111013230B1
:100F900011F48E7F01C081608093110102C021E0B5
:100FA00069C020E067C08A8110921C01311106C01F
:100FB00010921D018CE191E022E050C0353019F40F
:100FC000809324013DC03630A9F59B81913019F4FE
:100FD0008CEF97E704C0923041F48AEE97E7909344
:100FE00022018093210122E121C09330F1F481118B
:100FF00008C088E398E7909322018093210124E0C0
:1010000015C0813041F48CE198E7909322018093E0
:1010100021012CE10BC0823041F48EE098E79093DF
:101020002201809321012EE001C020E080E4809322
:10103000120118C0383079F0393031F4809326012C
:101040008CE191E020E00AC021E03A3009F020E094
:101050008CE191E003C086E291E021E090932201CF
:10106000809321012F3F31F447FD2E8180E880934A
:10107000120107C08F81811104C08E81821708F48C
:10108000282F209300017EC09091120197FF7AC013
:1010900090910E01E82E981708F4E92E9E1990936E
:1010A0000E01DD24D3949111D12CF12CFE1408F003
:1010B00066C020910C0180910F01909110012730A2
:1010C00078F08E010F5F1F4F68819C012F5F3F4FAB
:1010D0003093100120930F01F3D0F394E801E6CF91
:1010E0008115904708F04CC0F394F394F894E09184
:1010F0000F01F09110018991999121E00C01209349
:101100005700E8951124789480910F019091100177
:1011100002969093100180930F018F779927892B66
:1011200059F0DD2009F4C2CFFE1408F4BFCF80913E
:101130000D01882309F4BACFF894E0910F01F091E2
:101140001001329783E080935700E895789407B6B2
:1011500000FCFDCFF894E0910F01F091100132975F
:1011600085E080935700E895789407B600FCFDCFA2
:10117000F89481E180935700E895789497CFD11047
:1011800010920001109223018091010184FF6CC034
:10119000809100018F3F09F467C0F82E893010F06C
:1011A00028E0F22E8F19809300018091130198E8B6
:1011B000892780931301FF2009F449C0809112010F
:1011C00087FF27C080910E018F1508F4F82E8F1924
:1011D00080930E01E0900C01C4E1D1E084E191E044
:1011E000FC2FF81BFF1598F500910F0110911001CD
:1011F00086E08E1518F4C8015BD002C0F801849116
:10120000888321960F5F1F4F1093100100930F01E9
:10121000E5CFE0912101F091220186FF0BC084E12E
:1012200091E0DC0124912D9331962F2D280F2A1364
:10123000F9CF09C084E191E0DC0121912D932F2D9C
:10124000280F2A13FACFF0932201E09321016F2D8A
:1012500084E191E0ADDC84E08F0D8C3019F09FEFDC
:10126000909300018093010184E199B1947831F465
:101270008150D9F71092240110921E018091110122
:10128000803130F04E9B0FC080911101805109C018
:101290004E9909C080911101823028F0809111018E
:1012A00082508093110180911101811122CEF7CDDE
:1012B000F999FECF92BD81BDF89A992780B508951E
:1012C000262FF999FECF1FBA92BD81BD20BD0FB662
:1012D000F894FA9AF99A0FBE01960895F894FFCF00
:1012E000FF5A1E951400FA01DC0102C005900D9210
:1012F00021503040D8F70895CF93DF93CDB7DEB7B4
:10130000C058D1090FB6F894DEBF0FBECDBF84B769
:1013100014BE98E10FB6F8949093600010926000AC
:101320000FBE579AF89456985E9A209A219A559A29
:10133000539A5D9A83FDF1C0C0900001D0900101E5
:10134000E12CF12C6FEF7FEFCB01F701EC0DFD1DD0
:1013500044910E9448012FEFE21AF20AE114E0E101
:10136000FE0699F7603E764F8A4C924109F0B0C074
:10137000198280E090E0F601E80FF91F4591549141
:10138000FC01F059259134914217530719F081E07F
:10139000898305C00296811520E1920761F7898152
:1013A000882309F495C018E6C12E10E7D12EE12C50
:1013B000F12CB701A601407820E830E0CE0101967B
:1013C00092DFC701B6016856724F8F4F9F4F0AE4F4
:1013D00010E020E830E0AE014F5F5F4F0E94A600B2
:1013E00080E8C80ED11CE11CF11CE8E6CE16E2E74D
:1013F000DE06E104F104E9F6C12CB0E7DB2EE12CB6
:10140000F12C5601F0E7BF1A40E850E06FEF70E0B2
:10141000CE01019685D040910001509101014A0D05
:101420005B1D662757FD6095762F20E830E0CE01E2
:10143000019659DF0EE610E020E830E0AE014F5F84
:101440005F4FC701B6010E94A60020E8C20ED11C62
:10145000E11CF11CC11483E7D806E104F10489F60C
:10146000E12CA0E1FA2EEA18FB0840E850E06FEF0B
:1014700070E0CE01019654D09701E1E8EE16F10438
:1014800010F020E830E040910001509101014A0D38
:101490005B1D662757FD6095762FCE01019623DFF1
:1014A000B501705980E090E00AE410E020E830E0F7
:1014B000AE014F5F5F4F0E94A600F0E8AF0EB11C77
:1014C00020E8E21AF108A11480E1B80670F2299A26
:1014D000289A20E630E0C901880F991F820F931FD8
:1014E0000596009779F0EFE9FFE03197F1F700C03A
:1014F00000004E9905C05B984E9BFECF20E630E081
:101500000197EFCF8BB198E089278BB92150310932
:101510002115310501F70E945C015B9AA895FECF69
:10152000DC0101C06D9341505040E0F70895F894FC
:02153000FFCFEB
:02153200E602CF
:00000001FF
